:10000000370101002920A94873000000828096B8BA
:1000100022E44AE003457010218939E1B70900085C
:100020001309400F130A800F930480104A85812022
:10003000032540100D2852851D280325001025207A
:1000400003350010906088E090E4B6952A96333529
:10005000A600B386A50033F536012330C01079D54C
:100060002264026996BE8548730000008280914830
:10007000730000008280AD48730000008280930806
:10008000100873000000828093085008730000007D
:10009000828093087008730000008280732510C06E
:1000A0008280732500C0828093086008730000007E
:1000B00082800589F322008093920248B3E2A20075
:1000C00073900280828095487300000082809308BC
:1000D0000008730000008280A14873000000828045
:1000E0009308300873000000828093084008730072
:0C00F000000082800A4820000A4C20001A
:1001000001000000000000000000000000000000EE
:080110000000000000000000E7
:00000001FF
